:100000006F28B40014202008210403196A286420F2
:1000100084133408800664000D280E28A00A0319F2
:10002000A10F0B2880066A28FF3A841780056A28EA
:100030000F39A0000310A00DA00D1F08E039200407
:1000400001389F000030A10064303A209F149F18AF
:100050002728A1011E086A28A301A200FF30A207D9
:10006000031CA307031C6A280330A100DF303A20D9
:100070002E28A101E83EA000A109FC30031C432862
:10008000A00703184028A0076400A10F40282018EB
:100090004928A01C4D2800004D2808001030A80059
:1000A000A101A001A70CA60C031C5C282208A00734
:1000B00023080318230FA107A10CA00CA50CA40C66
:1000C000A80B522824086A28A009A109A00A03192C
:1000D000A10A080083130313831264000800831627
:1000E000FF239000831207309900831601309F0090
:1000F000093085008312850164302C2091208C20EA
:100100003908A10038083A20C830A000A101053004
:100110008400043001207E286400851D902808009A
:100120008C2800301820BA003A08A600A701FF303A
:10013000A200A3014E20B8002508B9000800630002
:020140009F28F6
:02400E00CC3FA5
:00000001FF
